:103DD10000010C01010402011E030A9604013205CF
:103DE100020206006407010108000009015A0E01E0
:103DF100010F000112006413010114013C1501FAC5
:103E01001664FA17FFFF1D00072000072400022790
:103E110001012F013C30010132010335FFFF36035F
:103E2100073CFFFF3DFFFF180002191E461A000262
:103E31001B00022D32C82E0001FAFAFA18000019EF
:103E4100FFFF1A00001B00002D32C82E0001FAFAF4
:103E5100FA18000019FFFF1A00001B00002DFFFFD8
:063E61002EFFFFFAFAFA41
:10004800900786E0FEA3E0FF7457BE0010D39F40E0
:100058000C903DD112001EE493F599804C90001449
:10006800E0D394044014900786E0FEA3E0FF903D9F
:10007800D112001EE493F599802F900014E0D394D8
:10008800034014900786E0FEA3E0FF903DE61200CF
:100098001EE493F5998012900786E0FEA3E0FF9096
:1000A8003DFB12001EE493F59990078612000E900E
:1000B8000786E0FEA3E0FF746C6F4E7003751300B3
:1000C80022900072E0B402087401900072F0D20C21
:1000D80090013AE090002AF090013BE090002BF06C
:1000E80090013CE090002CF0A20AB3401690013A2F
:1000F800E0700C90013BE0700690013CE0600280EB
:1001080002C20A90013AE0B4300F90013BE0B447D4
:100118000890013CE0643B60028004D20B8002C27C
:100128000BE557B40102800302024B900057E0F53B
:1001380065900062E0F567900063E0F568900074F0
:10014800E0F56990007AE0900029F090007CE0F5F5
:100158006490007DE0F566900080E0F56390008192
:10016800E0F562900090E0900041F0900091E090FE
:100178000042F0900092E0900043F0900093E090ED
:100188000044F0900094E0900045F0900095E090D5
:100198000046F0900096E0900047F0900097E090BD
:1001A8000048F0900099E0900033F090009AE090B9
:1001B8000034F090009BE0900035F090009CE090B7
:1001C8000036F0900079E0B4011790000A740FF03F
:1001D800A374FFF090000CE4F0A3F074029000798F
:1001E800F0900079E0B4035990000CE0FEA3E0FF22
:1001F80090000AE0FCA3E0FD1200037410123EE632
:100208007408123ED8EF900026F0EF700674FF9045
:100218000026F07400900079F090000BE090002721
:10022800F090000AE0900028F0900026E0900789FE
:10023800F0900027E090078AF0900028E090078B64
:10024800F0803F900081E07006755701756200A24A
:100258000AB3402E90013AE090002AF090013BE06A
:1002680090002BF090013CE090002CF090002AE0E8
:10027800700C90002BE0700690002CE06002800269
:10028800C20AE5657003756502E567700375670264
:100298007E887F75E5658E048F05FF123EC88C3811
:1002A8008D39E56875F0FAA4FFAEF0E5678E048F26
:1002B80005FF123EC88C3C8D3D90004FE0F55F90E5
:1002C800004DE0FE900069E0B5061890004CE0FE95
:1002D800900068E0B5060C90004BE0FE900059E0F5
:1002E8006E606F900069E07006900068E0600674C8
:1002F80000900059F0900069E0B402089000497439
:1003080001F08005900049E4F0900068E0B402082C
:1003180090004A7401F0800590004AE4F09000686B
:10032800E0600690004AE060028005755F03800384
:10033800755F04E558B55702D20C900068E090004C
:100348004CF0900069E090004DF0900059E090006A
:100358004BF0740090009EF0740090009FF07400C1
:100368009000A0F074009000A1F074009000A2F03A
:1003780074009000A3F074009000A4F07400900042
:10038800A5F074009000A6F074009000A7F0740027
:100398009000A8F074009000A9F074009000AAF0F2
:1003A80074009000ABF074009000ACF07400900002
:1003B800ADF074009000AEF074009000AFF07400DF
:1003C8009000B0F074009000B1F074009000B2F0AA
:1003D8007400900362F07401900363F0740090035A
:1003E80064F07400900365F07400900366F0740084
:1003F800900367F07400900368F074019003A2F012
:1004080074019003A3F074009003A4F074009003A7
:10041800A5F074009003A6F074009003A7F0740090
:100428009003A8F074019003E2F074009003E3F0E5
:1004380074009003E4F074009003E5F074009003F6
:10044800E6F074009003E7F074009003E8F074009D
:10045800900422F07400900423F07400900424F0B7
:100468007400900425F07400900426F07400900441
:1004780027F07400900428F022E5B554F7F5B5E5A7
:10048800B554FDF5B5C292C287C290C207E5B5540E
:10049800FBF5B5755004E55004F55190004FE0F5B3
:1004A8005F900025E4F0C209E5B554FEF5B5227564
:1004B8000A00750900AE09AF0A7457BE00039F50C1
:1004C80003020574903DD112001EE49390004E1271
:1004D8003EFE0FBF00010EE0FC903DD112001EEC65
:1004E800FEE493FFEEC39F5026AE09AF0A0FBF008C
:1004F800010E903DD112001EAE09AF0AE493FC90A4
:100508003DD112001EE49390004E123EFEECF0AE78
:1005180009AF0A903DD112001EE49390004E123E9E
:10052800FEE0FC903DD312001EECFCE493FDECD3FE
:100538009D4019903DD312001EE493FC903DD112CA
:10054800001EE49390004E123EFEECF0AE09AF0A96
:1005580074022FFF50010E8E098F0A780A74012643
:10056800F6500418E436F640030204BD22750A006A
:10057800750900AE09AF0A7415BE00039F50030247
:100588000642903E2812001EE49390004E123EFE52
:100598000FBF00010EE0FC903E2812001EECFEE4A6
:1005A80093FFEEC39F5026AE09AF0A0FBF00010E9E
:1005B800903E2812001EAE09AF0AE493FC903E2834
:1005C80012001EE49390004E123EFEECF0AE09AF0E
:1005D8000A903E2812001EE49390004E123EFEE060
:1005E800FC903E2A12001EECFCE493FDECD39D40E7
:1005F80019903E2A12001EE493FC903E2812001E19
:10060800E49390004E123EFEECF0AE09AF0A740F70
:100618006F4E7006750A15750900AE09AF0A7402A7
:100628002FFF50010E8E098F0A780A740126F650A2
:100638000418E436F6400302057B22750A007509A2
:1006480000AE09AF0A7415BE00039F5003020710DD
:10065800903E3D12001EE49390004E123EFE0FBFE6
:1006680000010EE0FC903E3D12001EECFEE493FFFC
:10067800EEC39F5026AE09AF0A0FBF00010E903E91
:100688003D12001EAE09AF0AE493FC903E3D1200F5
:100698001EE49390004E123EFEECF0AE09AF0A90B5
:1006A8003E3D12001EE49390004E123EFEE0FC9088
:1006B8003E3F12001EECFCE493FDECD39D401990E4
:1006C8003E3F12001EE493FC903E3D12001EE49350
:1006D80090004E123EFEECF0AE09AF0A740F6F4E5A
:1006E8007006750A15750900AE09AF0A74022FFF66
:1006F80050010E8E098F0A780A740126F6500418E4
:10070800E436F6400302064922750A00750900AE70
:1007180009AF0A7415BE00039F50030207DE903E1E
:100728005212001EE49390004E123EFE0FBF0001CD
:100738000EE0FC903E5212001EECFEE493FFEEC366
:100748009F5026AE09AF0A0FBF00010E903E52120D
:10075800001EAE09AF0AE493FC903E5212001EE45C
:100768009390004E123EFEECF0AE09AF0A903E5256
:1007780012001EE49390004E123EFEE0FC903E54A0
:1007880012001EECFCE493FDECD39D4019903E54FE
:1007980012001EE493FC903E5212001EE493900057
:1007A8004E123EFEECF0AE09AF0A740F6F4E7006A3
:1007B800750A15750900AE09AF0A74022FFF5001BA
:1007C8000E8E098F0A780A740126F6500418E4364A
:1007D800F6400302071722054C22054B22054DC29D
:1007E800CF2290F800E4936406600280FE758401CD
:1007F80075A70075FF80900788E4F075C91075A784
:100808000F75A1C775A70075D90075CEFF75A70F1D
:1008180075F1FE75F2FF75F33775F47875A4BA753E
:10082800A5FF75A60775AE0075AFFF75D48175D5A0
:10083800FF75D6FF75D7FFC293C294C291E5B55430
:10084800BFF5B5E5B554DFF5B5E5B554EFF5B5E554
:10085800B5547FF5B5E5B554F7F5B5E5B554FDF5EF
:10086800B575A70075A20175A14775F80975BC0192
:1008780075BE0475BD6C75BE0775BDA075BE0875DF
:10088800BD0175BC0075BB1875BC2075BA0875E844
:100898008075D11375A70F75E10575E20075C7401E
:1008A800759700759780740A123EB87597C0E597DA
:1008B8005420700280F8758F0275A700D2AF759822
:1008C8000075A90C75A70F75AB4375ADFB75AC1E0C
:1008D80075A700758911758E00758C00758A00D210
:1008E800A9D28C758D00758B00D2ABD28E75CD00D8
:1008F80075CC0075CA0075CB00D2ADC2CFD2CA750F
:1009080091047592007593CD75EF0675D94075CF32
:1009180001900786E4F0A3F0751300751400C299DE
:10092800D20A74C8F51875170012261975A70FE5AD
:10093800FB90001AF0E5FA90001BF0E5F990001C16
:10094800F075A70090F800E493F508122750122CD0
:100958008A900789E0900026F090078AE0900027A7
:10096800F090078BE0900028F090078CE090002929
:10097800F090078DE0F56590078EE0F56790078F9A
:10098800E0F568900790E0F569900791E0F56490CC
:100998000792E0F566900793E0F563900794E0F519
:1009A80062900795E090002AF0900796E090002B5F
:1009B800F0900797E090002CF0900798E0900041A5
:1009C800F0900799E0900042F090079AE090004379
:1009D800F090079BE0900044F090079CE090004561
:1009E800F090079DE0900046F090079EE090004749
:1009F800F090079FE0900048F09007A0E090003347
:100A0800F09007A1E0900034F09007A2E090003544
:100A1800F09007A3E0900036F07400900082F09008
:100A2800013AE0700C90013BE0700690013CE060F8
:100A3800028004C20A8002D20A90F807E493900068
:100A480021F0900021E0440A900021F0900021E07C
:100A580054FE900021F07406900012F07402900089
:100A680013F090F802E493900014F07403900015CA
:100A7800F07403900016F0741B900017F074059042
:100A88000018F0900014E0B404067404900018F004
:100A9800900014E0B403067403900018F0740490F6
:100AA8000019F090F804E49390001DF07400900091
:100AB8001EF090F805E49390001FF090F806E49378
:100AC800900020F074FF900022F0745A900125F0F5
:100AD8007446900126F07420900127F07434900138
:100AE80028F07448900129F0745090012AF074326B
:100AF80090012BF0743490012CF0742090012DF0AB
:100B0800743490012EF0742D90012FF074539001DD
:100B180030F0746F900131F0746C900132F07420F1
:100B2800900133F090007AE0D3940140067400906D
:100B3800007AF0755701755801740390004CF01253
:100B480000C91204B7900014E0B4040512064380EB
:100B580011900014E0D39404400512057580031227
:100B68000711122645E5B554FEF5B5900025E4F0C9
:100B7800900786E4F0A3F0752300752200754700FE
:100B880075290075280075480075310075300075A5
:100B98004900755300755400755900755004755116
:100BA8000175333C753200756F00756E007570CD38
:100BB80075550075560075420075430075440075FB
:100BC8004500755A00754600754100754000900053
:100BD80006E4F0A3F0900008E4F0A3F0755D00755A
:100BE8005E0090000E74FDF0A374E8F0900023E41A
:100BF800F07464900024F0C200D201C202D20375DE
:100C08004C00756C00C297C2A0C296C295C2A2C21F
:100C18000C7E017F00900028E0123EE6900027E05D
:100C28002FFF50010E90000AEEF0A3EFF09000267F
:100C3800E0700674FF900026F090000AE0FEA3E042
:100C4800FFEFD394FFEE940F400790000AE4F0A35F
:100C5800F07400900071F07400900079F0740090C6
:100C68000082F0740090008DF074009000B4F0E5FC
:100C7800667003756604743A90074EF074FD900729
:100C88004FF09003D4E0900414F0D2B0D2B7D2A7BA
:100C9800D2A6D2B1D2A3C207A2B6B39204A2B3B36A
:100CA8009205D29CD2EC75CF01A298B34005C298A8
:100CB800122FEEE5136006A299B3B340028005C275
:100CC80099123564E51464016005E514B4040280E2
:100CD800D5E54CD39405400CE559C394C85002059A
:100CE80059754C00E570C394F0501A786E12003FA5
:100CF800AE6EAF6FEFD394E8EE94034008057075BD
:100D08006F00756E00C28E7E047F00E54B123EE6D2
:100D1800E58D75F004A4FDACF0EF2DFDEE3CFCE58F
:100D28008B75F04084FF7E00ED2FFFEC3EFE8E2495
:100D38008F25D28EA2B6300401B35003020E74A2DE
:100D4800B6300401B35003020E74A2B6405A0553DC
:100D5800E5B54401F5B5900024E4F0E553D3956575
:100D680040447C887D75123CF08E228F23E5472F06
:100D7800FF50010E7401123ED88E228F238523471F
:100D8800755301C28E758D00758B00754B00D28E20
:100D98007403BE00039F50069000257401F0E542DD
:100DA800B40603754200D204A2B6B35003020E740F
:100DB800C20490006BE060181236A5A200B3400888
:100DC800E5B54408F5B58006E5B554F7F5B58002F4
:100DD800C20090006EE060181237FAA202B3400811
:100DE800E5B54402F5B58006E5B554FDF5B58006D0
:100DF800E5B554FDF5B5A207B34004D2968002C20A
:100E080096900059E06004D2958002C29590004AFD
:100E1800E0B40104D2978002C297900049E0B4017F
:100E280004D2A08002C2A0A209B34004D2A28002C8
:100E3800C2A2900018E0FE900014E0C39E40099002
:100E48000014E0D39408400974FB900023F01204C6
:100E58008190001DE0601590001DE0FE900017E0F5
:100E68006E600974FE900023F0120481C2CA7E01EC
:100E78007F00E54D123EE6E5CD2FFF50010E8E2690
:100E88008F27D2CAE564B4014890000EE0FCA3E0C5
:100E9800FDEFC39DEE9C4039B208E5294528601353
:100EA800A208B34008E5B54404F5B58006E5B55495
:100EB800FBF5B590000EE0FEA3E0FF900010E0FC0B
:100EC800A3E0FDEF2DFDEE3CFC90000EECF0A3ED51
:100ED800F0A2B3300501B35003020FB9A2B3300535
:100EE80001B35003020FB9A2B35003020FB2055465
:100EF800E5B54401F5B5900024E4F0E554D39567D1
:100F08005003020FB07CEA7D60AE26AF27123CF09A
:100F18008E288F29E568123EE674FF8E048F05FF40
:100F2800123EC88C288D29E5482DFD50010C74010E
:100F38008C068D07123ED88E288F29852948A2094C
:100F4800B340157464123EE6900067E08E048F0586
:100F5800FF123EC88C288D2975540190000EE0FEC2
:100F6800A3E0FFAC26AD2712000390000EEEF0A31D
:100F7800EFF0E566FF123EC8740AFF123EC8900003
:100F88007BE08C068D07123EE674148E048F05FFF5
:100F9800123EC8900010ECF0A3EDF0C2CA75CD0067
:100FA80075CC00754D00D2CAD205A2B3B34002C2B7
:100FB80005900025E0B40107E555C39406400302F7
:100FC80015C5E56C9025F8F8282873900059E0C3FA
:100FD80094024003021127E550D3940150030211F3
:100FE80027E55075F040A4FFAEF090031212001EE2
:100FF800E0C395445018E55075F040A4FFAEF0905A
:10100800031112001EE0F52D752C00021127E55082
:1010180075F040A4FFAEF090031012001EE0C395D7
:101028004440030210C3E55075F040A4FFAEF090B1
:10103800031112001EE55075F040A4FFAEF0E0FC6D
:1010480090030F12001EECFEE0FFEEC39FFEE5507A
:101058008E0475F040A4FFAEF090031012001EE05D
:10106800F40425448C0088F0A4FFAEF0E5508F040A
:101078008E0575F040A4FFAEF090031212001EE535
:101088005075F040A4FFAEF0E0FA90031012001E75
:10109800EAFEE0FFEEC39FFECDCCCD8E07123EC820
:1010A800E55075F040A4FFAEF090030F12001EE06B
:1010B8002DFD50010C8C2C8D2D8064E55075F04071
:1010C800A4FFAEF090030F12001EE55075F040A487
:1010D800FFAEF0E0FC90030E12001EECFEE0FFEE07
:1010E800C39F8544F0A4FFAEF0E5508F048E0575CC
:1010F800F040A4FFAEF090031012001EE0FECDCC2D
:10110800CD8E07123EC8E55075F040A4FFAEF090B2
:10111800030E12001EE02DFD50010C8C2C8D2D7538
:101128006C010215C5900059E0C3940240030212F5
:10113800DA90004FE0D395505003021283E55075C2
:10114800F040A4FFAEF090031812001EE0C39544CF
:101158005018E55075F040A4FFAEF0900317120048
:101168001EE0F52B752A00021283E55075F040A4A5
:10117800FFAEF090031612001EE0C3954440030230
:10118800121FE55075F040A4FFAEF090031712004F
:101198001EE55075F040A4FFAEF0E0FC9003151278
:1011A800001EECFEE0FFEEC39FFEE5508E0475F0D6
:1011B80040A4FFAEF090031612001EE0F40425448C
:1011C8008C0088F0A4FFAEF0E5508F048E0575F012
:1011D80040A4FFAEF090031812001EE55075F040D1
:1011E800A4FFAEF0E0FA90031612001EEAFEE0FF3C
:1011F800EEC39FFECDCCCD8E07123EC8E55075F0EC
:1012080040A4FFAEF090031512001EE02DFD500122
:101218000C8C2A8D2B8064E55075F040A4FFAEF04D
:1012280090031512001EE55075F040A4FFAEF0E0E3
:10123800FC90031412001EECFEE0FFEEC39F8544F1
:10124800F0A4FFAEF0E5508F048E0575F040A4FFC2
:10125800AEF090031612001EE0FECDCCCD8E071224
:101268003EC8E55075F040A4FFAEF090031412009C
:101278001EE02DFD50010C8C2A8D2BE550B4012267
:10128800E55FD39401401BE550C395555014E544E0
:10129800C39405500D90035FE0A828B8000695296F
:1012A80040028003755002E550B55F2290004FE080
:1012B800D395504019E55075F040A4FFAEF0900367
:1012C8001712001EE0A822B80006952340028002EB
:1012D800055F756C020215C5900059E0B4022AE555
:1012E8005075F040A4FFAEF090031712001EE0F511
:1012F8002B752A00E55075F040A4FFAEF090030E60
:1013080012001EE0F52D752C00900059E0B4030F73
:10131800900051E0F52B752A00752D00752C00758D
:101328006C030215C5E55075F040A4FFAEF09003BC
:101338002012001EE0C3955940030213FC90004997
:10134800E07036E550D394014029AE22AF23AC2C8F
:10135800AD2DEDD39FEC9E401AE55075F040A4FFEB
:10136800AEF090031E12001EE0A828B80005D39521
:10137800295002800215508034E550D39402402948
:10138800AE22AF23AC2CAD2DEDD39FEC9E401AE5D9
:101398005075F040A4FFAEF090031E12001EE0A8A6
:1013A80028B80005D39529500280021550E550C38E
:1013B800955F502FE550C395555028AE22AF23AC0A
:1013C8002AAD2BEFD39DEE9C4019E55075F040A453
:1013D800FFAEF090031F12001EE0A828B800069583
:1013E80029400280020550C290E55065516005C24F
:1013F80007755900756C040215C5E55075F040A4D1
:10140800FFAEF090031A12001EE0B40117E5507504
:10141800F040A4FFAEF090032012001EE0240AC39F
:10142800955940030214D2752F64752E00A207B394
:10143800500B900060E02405C3954440030214D289
:10144800E55075F040A4FFAEF090031D12001EE0B9
:10145800C395444064E55075F040A4FFAEF0900396
:101468001C12001EE55075F040A4FFAEF0E0FC90A1
:10147800031B12001EECFEE0FFEEC39F8544F0A4A0
:10148800FFAEF0E5508F048E0575F040A4FFAEF076
:1014980090031D12001EE0FECDCCCD8E07123EC873
:1014A800E55075F040A4FFAEF090031B12001EE05B
:1014B8002DFD50010C8C2E8D2FAE22AF23AC2EADFE
:1014C8002FEFD39DEE9C4002D207756C050215C51F
:1014D800E550B40109900059E0C394024003021595
:1014E800A5900358E0D3954450030215A5900356E0
:1014F800E0C395445040900357E0FE900355E0F454
:10150800042EFE900356E0F40425448E0088F0A4CF
:10151800FFAEF0900358E0FC900356E0F4042C8EE4
:10152800048F05FF123EC8900355E02DFD50010CB5
:101538008C2A8D2B802C900355E0FE900354E0F408
:10154800042E8544F0A4FFAEF0900356E08E048F7D
:1015580005FF123EC8900354E02DFD50010C8C2A63
:101568008D2BE550C3955F502FE550C395555028F6
:10157800AE22AF23AC2AAD2BEFD39DEE9C4019E5EC
:101588005075F040A4FFAEF090031F12001EE0A8B3
:1015980028B800069529400280037550029000493A
:1015A800E0B40106E550640160028003755002E56D
:0D15B8005065516005C207755900756C0043
:1025F800020FD302112D0212E002132D021402025F
:0226080014D8E4
:1015C500900050E02402A822B80007D395234002DA
:1015D500C207900025E0B40109900059E0C39403C7
:1015E500400302174B900049E0600302169BE5504B
:1015F500D394014034E55075F040A4FFAEF090035C
:101605001412001EE0A822B8001FD39523401AE546
:101615005075F040A4FFAEF090031F12001EE0A825
:1016250028B80005D39529500280021550E550D3FE
:101635009401402FE55075F040A4FFAEF0900312E1
:1016450012001EE0C39544501AE55075F040A4FF02
:10165500AEF090031E12001EE0A828B80005D39531
:1016650029500280021550E550D394014021E550E0
:10167500D39555401AE55075F040A4FFAEF09003A0
:101685001E12001EE0A828B80005D3952950028037
:10169500021550021740E550D394024034E55075C9
:1016A500F040A4FFAEF090031412001EE0A822B88B
:1016B500001FD39523401AE55075F040A4FFAEF006
:1016C50090031F12001EE0A828B80005D3952950E5
:1016D5000280021550E550D39402402FE55075F075
:1016E50040A4FFAEF090031212001EE0C3954450D3
:1016F5001AE55075F040A4FFAEF090031E12001ECF
:10170500E0A828B80005D39529500280021550E5B8
:1017150050D394024021E550D39555401AE55075B4
:10172500F040A4FFAEF090031E12001EE0A828B8FA
:101735000005D39529500280021550E5506551608A
:1017450005C207755900900060E0D3954450099093
:101755000054E0C395445002C207900059E070035D
:101765000219AEA2A5B34008A2A4B340030219977B
:10177500AE34AF357441D39F749C9E4005783412C6
:10178500003FAE34AF35EFB48806EEB413028003E4
:10179500021974A2A55003021837900059E0B4014C
:1017A5000B90004FE0D3955F4002055F900059E034
:1017B500B40253E55075F040A4FFAEF0900320123B
:1017C500001EE0C39559503E90004FE0D395504020
:1017D50020E550C395555019E55075F040A4FFAE6E
:1017E500F090031412001EE0A822B80006952340CD
:1017F500028002055090004FE0F55FE550655160AD
:1018050005C207755900900059E0B4032590004FB3
:10181500E0D395504007E550C39555400280020539
:101825005090004FE0F55FE55065516005C20775C2
:101835005900A2A45003021974900059E0B4016E36
:10184500900049E07035E550D394014029E5507585
:10185500F040A4FFAEF090031E12001EE0A828B8C9
:10186500000FD39529400A155075590085505F80A2
:101875000385505F8003755F018033E550D3940283
:101885004029E55075F040A4FFAEF090031E12000C
:101895001EE0A828B8000FD39529400A15507559A0
:1018A5000085505F800385505F8003755F0290005F
:1018B50059E0D394015003021968E55075F040A42E
:1018C500FFAEF090032012001EE0C39559400302BD
:1018D5001968900049E07041E550D394014034E522
:1018E5005075F040A4FFAEF090031112001EE0A861
:1018F50022B8001FD39523401AE55075F040A4FF88
:10190500AEF090031E12001EE0A828B80005D3957E
:1019150029500280021550803FE550D3940240348F
:10192500E55075F040A4FFAEF090031112001EE0E3
:10193500A822B8001FD39523401AE55075F040A49E
:10194500FFAEF090031E12001EE0A828B80005D3D4
:101955009529500280021550E55065516005C20772
:10196500755900E555B40704055D8003755D00E50F
:1019750062B4010EAE34AF35EF64407005EE649C81
:101985006002800EA2A54003755701A2A44003750D
:101995005702A2A5B3B35006A2A4B3B34002800672
:1019A500753500753400021A9CA2A5B34008A2A49F
:1019B500B34003021A88AE34AF357441D39F749C8B
:1019C5009E4005783412003FAE34AF35EFB488063B
:1019D500EEB413028003021A88A2A5406F90006836
:1019E500E0605A90004AE0B4010790004AE4F080B4
:1019F5000690004A7401F090004AE07005755F0397
:101A05008003755F0490004AE0B40104D297800218
:101A1500C297E550B4041AE55075F040A4FFAEF046
:101A250090031E12001EE0A828B80005D395295082
:101A3500028008755003C2077559008003755F045D
:101A4500E555B40704055D8003755D00A2A4403328
:101A5500900069E06021900049E0B40107900049D9
:101A6500E4F080069000497401F0900049E0B4016B
:101A750004D2A08002C2A0E555B40704055D800329
:101A8500755D00A2A5B3B35006A2A4B3B34002800E
:101A950006753500753400E5576558600690008277
:101AA500E06003021C24C29C751400751300C2CAB1
:101AB500E55790260AF82828738012122C8A800D83
:0D1AC500122D638008122E3C8003122F1595
:0F260A00021ABE021AC0021AC5021ACA021ACF59
:101AD200900029E090007AF0E565900057F0E56704
:101AE200900062F0E568900063F0E569900074F0A0
:101AF200E56490007CF0E56690007DF0E56390007F
:101B020080F0E562900081F090002AE090013AF0C6
:101B120090002BE090013BF090002CE090013CF013
:101B2200900041E0900090F0900042E0900091F02F
:101B3200900043E0900092F0900044E0900093F017
:101B4200900045E0900094F0900046E0900095F0FF
:101B5200900047E0900096F0900048E0900097F0E7
:101B6200900033E0900099F0900034E090009AF0F9
:101B7200900035E090009BF0900036E090009CF0E1
:101B82007400900082F0745A900125F0744690011E
:101B920026F07420900127F07434900128F07448E4
:101BA200900129F0745090012AF0743290012BF0C8
:101BB200743490012CF0742090012DF07434900153
:101BC2002EF0742D90012FF07453900130F0746F49
:101BD200900131F0746C900132F07420900133F076
:101BE2009003D4E0900414F0743A90074EF074FD20
:101BF20090074FF01200C9900004E4F0A3F09000A7
:101C0200067475F0A37430F09000087475F0A37434
:101C120030F0855758D2CA754B00D29C741B900085
:101C220023F0E555C394065005E550B55102804EA8
:101C3200C207E55075F040A4FFAEF09003221200F7
:101C42001EE030E003D38001C39293E55075F0406B
:101C5200A4FFAEF090032312001EE030E003D38015
:101C620001C39294855051AE28AF297405BE00037A
:101C72009F5007E544D3940550028002D290E55567
:101C8200D394055003021D45C207E550D394014089
:101C920059E55075F040A4FFAEF090031E12001EED
:101CA200E0A828B80007D3952940021550E55065F1
:101CB200516035E55075F040A4FFAEF0900322125A
:101CC200001EE030E003D38001C39293E55075F02B
:101CD20040A4FFAEF090032312001EE030E003D3D5
:101CE2008001C392948550518059E555B4061A90EB
:101CF20000ACE030E003D38001C392939000ADE0EA
:101D020030E003D38001C39294E555B40716AE28A0
:101D1200AF297404BE00039F5006C293D29480047C
:101D2200D293C294E555B4081A90009EE030E003C5
:101D3200D38001C3929390009FE030E003D38001EF
:101D4200C39294900072E06058E54475F00284FFFB
:101D52007E0090014E12001EE0F55BE54675F00A2A
:101D620084FF7E0090024E12001EE0F55CE55B25CA
:101D72005CD39464400BE55B255CC39464F55B80A3
:101D820003755B00E55B75F00284FF7E008F5BEFFD
:101D9200C394335007EF24CDF55B8003755BFF805E
:101DA2001CE54475F00284FF7E0090014E12001E75
:101DB200E075F00284FF7E00EF24CDF55BE595C36C
:101DC200955B4004C2928002D292A207B34005E51D
:101DD20055B407037570CDE595C395704004C2876D
:101DE2008002D287E542C3940640030223E9A2EDB2
:101DF200B350030223E9C2EDE5426003021F4B7EAA
:101E0200017F00E5BE123EE6E5BD2FFF50010E90B8
:101E12000000EEF0A3EFF0900029E0B401177E0F6E
:101E22007FFF900000E0FCA3E0FD120003900000A1
:101E3200EEF0A3EFF0900079E0B4025B900000E0D6
:101E4200FEA3E0FF90000AE0FCA3E0FDEDD39FECCF
:101E52009E400F900000E0F8A3E090000AC8F0A3B3
:101E6200C8F0900000E0FEA3E0FF90000CE0FCA3AD
:101E7200E0FDEFD39DEE9C400F900000E0F8A3E060
:101E820090000CC8F0A3C8F0900000E0FEA3E0FFB1
:101E92007404123ED88F43900079E0706090000085
:101EA200E0FEA3E0FF90000AE0FCA3E0FDEFD39D7B
:101EB200EE9C400D120003900000EEF0A3EFF080C4
:101EC20007900000E4F0A3F0900000E0FEA3E0FF22
:101ED2007410123EE6900026E08E048F05FF123E3B
:101EE200C8900000ECF0A3EDF07400D39D74019C47
:101EF2004008900001E0F54380037543FFE5437518
:101F0200F00AA4FFAEF074198E048F05FF123EC8CA
:101F12008D44ED2531FFAE3050010E7401123ED8D2
:101F22008F44854431753000EFD394624003754489
:101F320062900072E064016006900066E0600280D8
:101F420005754201800375BB17E542B401028003A7
:101F520002203B7E017F00E5BE123EE6E5BD2FFF7B
:101F620050010E900000EEF0A3EFF0900072E0B48A
:101F7200017EE53345326025AC32AD331DBDFF0134
:101F82001C8F028E038C068D07903A1C12002EE4E1
:101F920093FE740193FFEFC39AEE9B400280057893
:101FA20032123F10AE32AF3374B3BE0025D39F401E
:101FB20021900000E0FCA3E0FD0FBF00010E903A6B
:101FC2001C12002EE493FE740193FFEDC39FEC9E5E
:101FD20040028005783212003FAE32AF33E569121B
:101FE2003EE674648E048F05FF123EC88D46803330
:101FF200900066E0602D900000E0FEA3E0FFEFD3CA
:102002009400EE9408400F900066E0B40104C20907
:102012008002D209800D900066E0B40104D20980EA
:1020220002C209900072E064026006900066E060FD
:102032000575BB168003754202E542B402028003B5
:102042000221297E017F00E5BE123EE6E5BD2FFF9B
:1020520050010E900000EEF0A3EFF0900072E0B499
:10206200027EE53345326025AC32AD331DBDFF0142
:102072001C8F028E038C068D07903B8612002EE485
:1020820093FE740193FFEFC39AEE9B4002800578A2
:1020920032123F10AE32AF3374B3BE0025D39F402D
:1020A20021900000E0FCA3E0FD0FBF00010E903B79
:1020B2008612002EE493FE740193FFEDC39FEC9E03
:1020C20040028005783212003FAE32AF33E569122A
:1020D2003EE674648E048F05FF123EC88D4680333F
:1020E200900066E0602D900000E0FEA3E0FFEFD3D9
:1020F2009400EE9408400F900066E0B40104C20917
:102102008002D209800D900066E0B40104D20980F9
:1021120002C209900072E07003754600900066E00A
:102122007002C20975BB1FE542B403457E017F0000
:10213200E5BE123EE6E5BD2FFF50010E900000EE17
:10214200F0A3EFF07409123EE674E68E048F05FFE9
:10215200123EC88C408D41E5492DFD50010C7401A1
:102162008C068D07123ED88E408F4185414975BB42
:1021720019E542B4040280030222D17E017F00E508
:10218200BE123EE6E5BD2FFF50010E900000EEF0BC
:10219200A3EFF07404123ED88F4AE563B4010280C3
:1021A2000302225E756A00756A00E56AD3940740ED
:1021B2000302224BE56A900041123EFEE0D3954AAB
:1021C200501AE56A900041123EFEE0F404254AFEF0
:1021D200E56A900037123EFEEEF08017E56A900045
:1021E20041123EFEE0C3954AFEE56A900037123E78
:1021F200FEEEF0E56AC394044009900084E0C395C2
:102202006A503BE56A6029E56A900037123EFEFE9D
:10221200E0FFEE90003FE0D39F4013E56A90003765
:10222200123EFEE090003FF0E56A900040F0800E22
:10223200900037E090003FF07400900040F0786A20
:10224200740126F640030221AC900040E0F404241D
:1022520008F555E555D394054002C290E563D39441
:1022620001402FE54AD3946E4004D20D8002C20D84
:10227200755505E563B40205A20DB34002800375EE
:102282005507E563B40306A20DB3B340028003759C
:102292005507E55665556008E55004F551855556D4
:1022A200E555B40708E5B54480F5B58006E5B554B3
:1022B2007FF5B5E55564066005E555B40808E5B552
:1022C2004410F5B58006E5B554EFF5B575BB13E5D9
:1022D20042B4050280030223E57E017F00E5BE12BF
:1022E2003EE6E5BD2FFF50010E900000EEF0A3EF99
:1022F200F07404123ED88F45E562B40202800302F4
:1023020023E2756A00756A00E56AD394034003020A
:102312002399E56A900033123EFEE0D39545501AA8
:10232200E56A900033123EFEE0F4042545FEE56ABC
:1023320090002D123EFEEEF08017E56A90003312F7
:102342003EFEE0C39545FEE56A90002D123EFEEE8C
:10235200F0E56A6029E56A90002D123EFEFEE0FF7C
:10236200EE900031E0D39F4013E56A90002D123EBB
:10237200FEE0900031F0E56A900032F0800E9000AD
:102382002DE0900031F07400900032F0786A740110
:1023920026F6400302230A900082E07043E52945B5
:1023A200286036E557C39403500A900032E004C314
:1023B200940340028007900032E004F557E557D3BA
:1023C2009402400A900032E004D394025002800743
:1023D200900032E004F5578007900032E004F55790
:1023E20075BB180542D2ECE55DD394045003022478
:1023F200D175CF01C292AE34AF357488D39F7413B6
:102402009E4005A2A5B34014AE34AF357488D39F65
:1024120074139E4005A2A4B340028048783412008F
:102422003FAE34AF35EFB4883BEEB41337A2A5B359
:10243200500990004FE0D39550500280040550801F
:1024420011A2A5B3500890004FE0655060028002CF
:10245200D207A2A4B35007E550D3940150028004DE
:102462001550C207A2A5B3B35006A2A4B3B340024B
:102472008006753500753400E55065516035E550CC
:1024820075F040A4FFAEF090032212001EE030E08F
:1024920003D38001C39293E55075F040A4FFAEF0E0
:1024A20090032312001EE030E003D38001C3929414
:1024B200855051A20740057570CD80037570FFE508
:1024C20095C395704004C2878002D2870223F3AE7F
:1024D20024AF25EFD39420EE944E50030225CC1264
:1024E2000481C28E758D00758B00754B00D28EC231
:1024F20007756F00756E007570CD755004752300F9
:10250200752200755300755900C296900059E0601B
:1025120004D2958002C29590004AE0B40104D29799
:102522008002C297900049E0B40104D2A08002C2A6
:10253200A0A209B34004D2A28002C2A290006BE022
:1025420060181236A5A200B34008E5B54408F5B5F7
:102552008006E5B554F7F5B58002C20090006EE042
:1025620060181237FAA202B34008E5B54402F5B585
:102572008006E5B554FDF5B58006E5B554FDF5B523
:1025820090000E74FDF0A374E8F0E542B406037502
:102592004200900025E4F0752500752400758D0039
:1025A200758B00754B00900024E0C3940350089093
:1025B2000024E004F080067403900024F0900024CC
:1025C200E0B40306E5B554FEF5B5AE26AF27EFD36A
:1025D2009410EE9427401CC2CA75CD0075CC0075CC
:1025E2002700752600D2CA754D007529007528008E
:0625F200755400020CAE5E
:1039AC00000001000132016401960196020002122E
:1039BC0002240200020003000340038003C0040041
:1039CC000440048004C00500060006000600060042
:1039DC00060006000600060000FF01310163019598
:1039EC0001FF01FF0211022302FF02FF02FF033F4E
:1039FC00037F03BF03FF043F047F04BF04FF05FFE5
:103A0C0006FF06FF06FF06FF06FF06FF06FF06FF82
:103A1C000FAA0FA50F9F0F9A0F940F8D0F870F8072
:103A2C000F780F710F680F600F570F4E0F450F3B3C
:103A3C000F300F250F1A0F0E0F020EF50EE80EDBCE
:103A4C000ECC0EBE0EAE0E9F0E8E0E7D0E6C0E5A52
:103A5C000E470E340E200E0C0DF70DE20DCB0DB5EE
:103A6C000D9D0D850D6D0D540D3A0D200D050CE9B8
:103A7C000CCE0CB10C940C760C580C3A0C1B0BFBAA
:103A8C000BDB0BBB0B9A0B790B570B350B130AF19A
:103A9C000ACE0AAB0A870A640A400A1C09F809D440
:103AAC0009B0098C09670943091F08FB08D608B23D
:103ABC00088E086A0846082307FF07DC07B9079633
:103ACC0007730751072F070D06EC06CA06AA0689CD
:103ADC0006690649062A060A05EC05CD05B00592CD
:103AEC0005750558053C0520050504EA04CF04B509
:103AFC00049C04820469045104390422040B03F469
:103B0C0003DE03C803B2039D038903750361034DF0
:103B1C00033B03280316030402F202E102D102C0A4
:103B2C0002B002A00291028202730265025702499E
:103B3C00023C022F02220216020901FD01F201E6EB
:103B4C0001DB01D001C601BB01B101A7019D0194AC
:103B5C00018B0182017901700168016001580150EB
:103B6C000148014101390132012B0125011E0118C7
:103B7C000111010B010500FF00FA0FA60FA00F9910
:103B8C000F920F8B0F840F7C0F740F6B0F620F58FB
:103B9C000F4E0F430F380F2C0F1F0F120F050EF780
:103BAC000EE80ED80EC80EB70EA50E930E800E6C36
:103BBC000E580E420E2C0E150DFD0DE40DCB0DB155
:103BCC000D950D790D5D0D3F0D200D010CE10CC017
:103BDC000C9E0C7C0C590C350C100BEA0BC40B9E78
:103BEC000B760B4F0B260AFD0AD40AAA0A800A553B
:103BFC000A2A09FF09D409A8097C0950092508F9E2
:103C0C0008CD08A10875084A081E07F307C8079DC8
:103C1C0007730749072006F706CE06A6067E065749
:103C2C000630060A05E405BF059B057705540532E9
:103C3C00051004EF04CE04AE048F04710453043554
:103C4C00041903FD03E203C703AD0394037B036371
:103C5C00034B0334031E030802F302DE02CA02B64E
:103C6C0002A30291027F026D025C024C023C022C08
:103C7C00021D020E020001F201E401D701CA01BECD
:103C8C0001B101A6019A018F0185017A01700166CB
:103C9C00015D0153014A0141013901310129012121
:103CAC0001190112010B010400FD00F700F000EAFC
:103CBC0000E400DE00D900D300CE00C900C400BF70
:103CCC0000BA00B500B100AD00A800A400A0009C93
:103CDC00009900950091008E008A00870084008175
:043CEC00007E007BDB
:10261900751A00751900AE19AF1AAC17AD18EDC3CC
:102629009FEC9E401674FF123EB875CF01781A745C
:102639000126F6500418E436F650DB22900786E4AA
:10264900F0A3F0751000750F00751300751400C222
:102659000ED20F22C2AF75D900758F0375B7A57554
:10266900B7F190F800E4F0758F0175B7A575B7F16A
:10267900E50890F800F075B7A575B7F190F801E491
:10268900F075B7A575B7F190079DE090F802F07560
:10269900B7A575B7F19007A1E090F803F075B7A554
:1026A90075B7F190079EE090F804F075B7A575B776
:1026B900F190079FE090F805F075B7A575B7F1900F
:1026C90007A0E090F806F075B7A575B7F19007A2D5
:1026D900E090F807F0758F0075D940D2AF229007C6
:1026E90088E0B4AB61C2AF75D90075B62275F52221
:1026F900758F0375B7A575B7F1740090F600F0757D
:102709008F01750A00750900AE09AF0A7413BE007E
:10271900279F402475B7A575B7F190078912001E48
:10272900E0FC90F60012001EECF0780A740126F61F
:10273900500418E436F650D0758F0075F51175B64A
:102749002075D940D2AF22C2AF75D90075F522756F
:102759000A00750900AE09AF0A7413BE00229F4032
:102769001F90F60012001EE493FC90078912001EC8
:10277900ECF0780A740126F6500418E436F650D5C0
:1027890075F51175D940D2AF22900788E0B4AA0235
:1027990080030228CFC2AF75D90075B62275F5221C
:1027A900758F0375B7A575B7F1740090EE00F075D4
:1027B900B7A575B7F1740090F000F075B7A575B7B6
:1027C900F1740090F200F075B7A575B7F174009037
:1027D900F400F0758F01750A00750900AE09AF0A9A
:1027E90074FFC39F74019E402475B7A575B7F19016
:1027F900004E12001EE0FC90EE0012001EECF07874
:102809000A740126F6500418E436F650CF750A000A
:10281900750900AE09AF0A74FFC39F74019E402475
:1028290075B7A575B7F190024E12001EE0FC90F045
:102839000012001EECF0780A740126F6500418E420
:1028490036F650CF750A00750900AE09AF0A74FF54
:10285900C39F74019E402475B7A575B7F190044EC6
:1028690012001EE0FC90F20012001EECF0780A74CF
:102879000126F6500418E436F650CF750A0075099A
:1028890000AE09AF0A74FFC39F74019E402475B757
:10289900A575B7F190064E12001EE0FC90F40012E7
:1028A900001EECF0780A740126F6500418E436F696
:1028B90050CF758F0075F51175B62075D940D2AF17
:1028C900743A90074EF022900788E0B4AA02800378
:1028D900022A0DC2AF75D90075B62275F522758F1A
:1028E9000375B7A575B7F1740090E600F075B7A543
:1028F90075B7F1740090E800F075B7A575B7F17474
:102909000090EA00F075B7A575B7F1740090EC0076
:10291900F0758F01750A00750900AE09AF0A74FFD9
:10292900C39F74019E402475B7A575B7F190004EF9
:1029390012001EE0FC90E60012001EECF0780A740A
:102949000126F6500418E436F650CF750A007509C9
:1029590000AE09AF0A74FFC39F74019E402475B786
:10296900A575B7F190024E12001EE0FC90E8001226
:10297900001EECF0780A740126F6500418E436F6C5
:1029890050CF750A00750900AE09AF0A74FFC39FDD
:1029990074019E402475B7A575B7F190044E1200D5
:1029A9001EE0FC90EA0012001EECF0780A74012681
:1029B900F6500418E436F650CF750A00750900AED2
:1029C90009AF0A74FFC39F74019E402475B7A575AA
:1029D900B7F190064E12001EE0FC90EC0012001EAA
:1029E900ECF0780A740126F6500418E436F650CF54
:1029F900758F0075F51175B62075D940D2AF743A47
:102A090090074EF022900788E0B4AA028003022BB7
:102A19004BC2AF75D90075B62275F522758F03754E
:102A2900B7A575B7F1740090DE00F075B7A575B755
:102A3900F1740090E000F075B7A575B7F1740090D6
:102A4900E200F075B7A575B7F1740090E400F07570
:102A59008F01750A00750900AE09AF0A74FFC39F9B
:102A690074019E402475B7A575B7F190004E120008
:102A79001EE0FC90DE0012001EECF0780A740126BC
:102A8900F6500418E436F650CF750A00750900AE01
:102A990009AF0A74FFC39F74019E402475B7A575D9
:102AA900B7F190024E12001EE0FC90E00012001EE9
:102AB900ECF0780A740126F6500418E436F650CF83
:102AC900750A00750900AE09AF0A74FFC39F740146
:102AD9009E402475B7A575B7F190044E12001EE00B
:102AE900FC90E20012001EECF0780A740126F65000
:102AF9000418E436F650CF750A00750900AE09AF1F
:102B09000A74FFC39F74019E402475B7A575B7F178
:102B190090064E12001EE0FC90E40012001EECF03C
:102B2900780A740126F6500418E436F650CF758FEA
:102B39000075F51175B62075D940D2AF743A900772
:102B49004EF022900788E0B4AA028003022C89C2C1
:102B5900AF75D90075B62275F522758F0375B7A5BE
:102B690075B7F1740090D600F075B7A575B7F17413
:102B79000090D800F075B7A575B7F1740090DA0028
:102B8900F075B7A575B7F1740090DC00F0758F0189
:102B9900750A00750900AE09AF0A74FFC39F740175
:102BA9009E402475B7A575B7F190004E12001EE03E
:102BB900FC90D60012001EECF0780A740126F6503B
:102BC9000418E436F650CF750A00750900AE09AF4E
:102BD9000A74FFC39F74019E402475B7A575B7F1A8
:102BE90090024E12001EE0FC90D80012001EECF07C
:102BF900780A740126F6500418E436F650CF750A9F
:102C090000750900AE09AF0A74FFC39F74019E40A5
:102C19002475B7A575B7F190044E12001EE0FC901B
:102C2900DA0012001EECF0780A740126F650041836
:102C3900E436F650CF750A00750900AE09AF0A747B
:102C4900FFC39F74019E402475B7A575B7F190061F
:102C59004E12001EE0FC90DC0012001EECF0780A17
:102C6900740126F6500418E436F650CF758F0075B6
:102C7900F51175B62075D940D2AF743A90074EF068
:102C890022C2AF75D90075F522750A00750900AE23
:102C990009AF0A74FFC39F74019E401F90EE001292
:102CA900001EE493FC90004E12001EECF0780A74AA
:102CB9000126F6500418E436F650D4750A00750951
:102CC90000AE09AF0A74FFC39F74019E401F90F0C4
:102CD9000012001EE493FC90024E12001EECF078E4
:102CE9000A740126F6500418E436F650D4750A0021
:102CF900750900AE09AF0A74FFC39F74019E401F96
:102D090090F20012001EE493FC90044E12001EEC97
:102D1900F0780A740126F6500418E436F650D47592
:102D29000A00750900AE09AF0A74FFC39F74019EBA
:102D3900401F90F40012001EE493FC90064E12000E
:102D49001EECF0780A740126F6500418E436F650A1
:102D5900D475F51175D940D2AF22C2AF75D90075B6
:102D6900F522750A00750900AE09AF0A74FFC39F01
:102D790074019E401F90E60012001EE493FC90002F
:102D89004E12001EECF0780A740126F6500418E47D
:102D990036F650D4750A00750900AE09AF0A74FFFA
:102DA900C39F74019E401F90E80012001EE493FC2B
:102DB90090024E12001EECF0780A740126F65004B7
:102DC90018E436F650D4750A00750900AE09AF0A41
:102DD90074FFC39F74019E401F90EA0012001EE415
:102DE90093FC90044E12001EECF0780A740126F64A
:102DF900500418E436F650D4750A00750900AE0976
:102E0900AF0A74FFC39F74019E401F90EC0012002B
:102E19001EE493FC90064E12001EECF0780A740131
:102E290026F6500418E436F650D475F51175D940D4
:102E3900D2AF22C2AF75D90075F522750A0075099E
:102E490000AE09AF0A74FFC39F74019E401F90DE54
:102E59000012001EE493FC90004E12001EECF07864
:102E69000A740126F6500418E436F650D4750A009F
:102E7900750900AE09AF0A74FFC39F74019E401F14
:102E890090E00012001EE493FC90024E12001EEC2A
:102E9900F0780A740126F6500418E436F650D47511
:102EA9000A00750900AE09AF0A74FFC39F74019E39
:102EB900401F90E20012001EE493FC90044E1200A1
:102EC9001EECF0780A740126F6500418E436F65020
:102ED900D4750A00750900AE09AF0A74FFC39F745F
:102EE900019E401F90E40012001EE493FC90064EE0
:102EF90012001EECF0780A740126F6500418E43624
:102F0900F650D475F51175D940D2AF22C2AF75D933
:102F19000075F522750A00750900AE09AF0A74FF3C
:102F2900C39F74019E401F90D60012001EE493FCBB
:102F390090004E12001EECF0780A740126F6500437
:102F490018E436F650D4750A00750900AE09AF0ABF
:102F590074FFC39F74019E401F90D80012001EE4A5
:102F690093FC90024E12001EECF0780A740126F6CA
:102F7900500418E436F650D4750A00750900AE09F4
:102F8900AF0A74FFC39F74019E401F90DA001200BC
:102F99001EE493FC90044E12001EECF0780A7401B2
:102FA90026F6500418E436F650D4750A007509005F
:102FB900AE09AF0A74FFC39F74019E401F90DC00E5
:102FC90012001EE493FC90064E12001EECF0780AE3
:102FD900740126F6500418E436F650D475F51175C7
:102FE900D940D2AF22E51464046006E59964FF6014
:102FF900028031A20E4004D20E8027E514600874C5
:10300900E62514900023F0E513600874F025139069
:103019000023F0E514B4010280FE75140075130055
:10302900C20E8002C20EE51490394FF82828737534
:103039001400E599B4FF03751301E599B4FE03750E
:103049001302E599B4FD03751303E599B4FC0375FF
:103059001304E599B4FA03751305E599B4FB0675EC
:103069001401120481E599B4F90675140412048156
:10307900E599D394E54007E599C394F04002801699
:103089008599157514027E017F00E515C394E61232
:103099003EE68E0D8F0E900786E4F0A3F0E599D3F6
:1030A90094C44007E599C394E640028028859915A0
:1030B90075140374E5C39515F50E750D00AE0DAFC6
:1030C9000E9039AC12002EE493F8740193900786A0
:1030D900C8F0A3C8F0D299023563900786E0FEA331
:1030E900E0FFEFC39400EE94054009EFD394FFEE9F
:1030F90094064013900786E0FEA3E0FF90004E126D
:10310900001EE599F0800385996B90078612000EE1
:10311900900786E0FEA3E0FFEFB40106EEB40702D4
:10312900800302337090074EE0B43C0280030233FF
:103139007075FFA0A20AB35005A20BB34003023277
:1031490063C29C90007AE090078CF0900057E09061
:10315900078DF0900062E090078EF0900063E09098
:10316900078FF0900074E0900790F090007CE09059
:103179000791F090007DE0900792F0900080E09038
:103189000793F0900081E0900794F090013AE09065
:103199000795F090013BE0900796F090013CE09094
:1031A9000797F0900090E0900798F0900091E090D8
:1031B9000799F0900092E090079AF0900093E090C0
:1031C900079BF0900094E090079CF0900095E090A8
:1031D900079DF0900096E090079EF0900097E09090
:1031E900079FF0900099E09007A0F090009AE09076
:1031F90007A1F090009BE09007A2F090009CE0905E
:1032090007A3F07400900082F01200C974AB900714
:0D32190088F01226E774AA900788F0E557A8
:06394F000230380230E3F3
:10322600903970F82828738012122792800D122880
:0B323600D08008122A0E8003122B4CDF
:0F39700002322D02322F02323402323902323E3D
:10324100900788E4F090013AE0700C90013BE07047
:103251000690013CE060028004C20A8002D20A02A8
:103261003365C29C900078E0900789F090005EE0A1
:1032710090078AF090005FE090078BF090007AE071
:1032810090078CF0900057E090078DF0900062E07D
:1032910090078EF0900063E090078FF0900074E04B
:1032A100900790F090007CE0900791F090007DE015
:1032B100900792F0900080E0900793F0900081E0F9
:1032C100900794F090013AE0900795F090013BE06F
:1032D100900796F090013CE0900797F0900090E005
:1032E100900798F0900091E0900799F0900092E09B
:1032F10090079AF0900093E090079BF0900094E083
:1033010090079CF0900095E090079DF0900096E06A
:1033110090079EF0900097E090079FF0900099E051
:103321009007A0F090009AE09007A1F090009BE038
:103331009007A2F090009CE09007A3F07400900029
:1033410082F074AB900788F01226E774AA90078880
:10335100F01227921228D0122A0E122B4CD29C75F1
:1033610099FB80FED29C7514007513007599FB02C0
:103371003563900786E0FEA3E0FFEF4E7006859966
:1033810010750F00900786E0FEA3E0FF74016F4EF9
:10339100701BAC0FAD10AA0DAB0EED2BFBEC3AFA86
:1033A1008A068B0790004E12001EE599F090078661
:1033B10012000E900786E0FEA3E0FF74026F4E70CC
:1033C1000C1200C985159975140075130002356337
:1033D100900786E0FEA3E0FF90004E12001EE599E3
:1033E100F090078612000E900786E0FEA3E0FFAC86
:1033F1000DAD0E8F028E038C068D079039E41200FD
:103401002EE493F9740193FEEAD39EEB994009856A
:103411001599751400751300023563900786E0FE57
:10342100A3E0FF90004E12001EE599F0900786126E
:10343100000E900786E0FEA3E0FFEFB40006EEB4B5
:103441000102800302356375FFA090001CE0D39454
:10345100C7400B90001CE0C394C8F516801A900079
:103461001CE0D39463400B90001CE0C39464F516F8
:10347100800690001CE0F516E51675F002A4FFAE7B
:10348100F08F6AEF90004E123EFEEFFCE0FDEC90F3
:103491000051123EFEEDFCE0FDEC2DB5160280035D
:1034A1000235550FEF90004E123EFEE56AFFE0FC3B
:1034B100EF900052123EFEECFFE0FCEFC39CB5160C
:1034C100028003023555E56A900050123EFEE56A1E
:1034D100FFE0FCEF900053123EFEECFFE0FCEF2C0E
:1034E100B51671E56A900054123EFEE0C395169040
:1034F100079DF0E56A900055123EFEE0C3951690D7
:10350100079EF0E56A900058123EFEE0C3951690C2
:10351100079FF0E56A900059123EFEE0C3951690B0
:1035210007A0F0E56A90005A123EFEE0C39516909E
:1035310007A1F0E56A90005B123EFEE0C39516908C
:1035410007A2F012265D7599F975186475170012B6
:10355100261980FE7599FF751864751700122619D2
:0235610080FEEA
:093955000233730233D102341C69
:1035630022E51390395EF82828730236A490078663
:10357300E0FEA3E0FF90001212001EE0F599900711
:103583008612000E900786E0FEA3E0FF74116F4ED3
:1035930070037513000236A48561990236A490075F
:1035A30086E0FEA3E0FF90004E12001EE0F599EFC7
:1035B300B40107EEB4070375130090078612000EDB
:0735C3000236A4900787E027
:0F395E0002356D02357002359B0235A10235C668
:1035CA0090397FF828287385239902369985299995
:1035DA000236998543990236998546990236998524
:1035EA005099023699855F9902369985559902361E
:1035FA0099855799023699756D00900069E07006B1
:10360A00900068E060028016A2A44006E56D4404BA
:10361A00F56DA2A54006E56D4402F56D801A90008D
:10362A004AE0B40106E56D4410F56D900049E0B436
:10363A000106E56D4420F56DA207B34006E56D4429
:10364A0001F56DA209B34006E56D4408F56D856D77
:10365A0099803CA20FB340077599FAC20F8017A24E
:10366A000CB3400575990F800B900023E0F59990F3
:10367A000023E4F0C20C80178541998012854A998B
:0F368A00800D85459980087599FC8003751300A4
:10397F000235D10235D70235DD0235E30235E902D2
:10398F0035EF0235F50235FB02360102365D0236A0
:0D399F008202368702368C0236910236967F
:0B36990090078612000E80031200480C
:03396D000236A17E
:1036A4002290006BE0B4010385231190006BE0B419
:1036B400020385291190006BE0B403038543119044
:1036C400006BE0B4040385461190006BE0B405037D
:1036D40085501190006BE0B4060385551190006B82
:1036E400E0B4070385571190006CE0FE90006DE094
:1036F400C39E500302377B90006BE0D39404402CAC
:1037040090006CE0D39511500990006DE0C39511C1
:1037140050028002D20090006CE0D39511500990C1
:10372400006DE0C395115002C200804990006BE027
:10373400B4041890006DE0C395115002D2009000BB
:103744006CE0D395114002C200802A90006CE0C363
:103754009511500990006DE0D3951150028002D26A
:103764000090006CE0D39511500990006DE0C39572
:10377400115002C200807E90006BE0D39404402C70
:1037840090006CE0C39511400990006DE0D3951151
:1037940040028002C20090006CE0C3951140099081
:1037A400006DE0D395114002D200804990006BE097
:1037B400B4041890006CE0C395115002C20090004C
:1037C4006DE0D395114002D200802A90006CE0C3D2
:1037D4009511400990006DE0D395114002D20090FC
:1037E400006CE0D39511400990006DE0C395114041
:1037F400028002C2002290006EE0B401038523110E
:1038040090006EE0B4020385291190006EE0B403C9
:103814000385431190006EE0B404038546119000C3
:103824006EE0B4050385501190006EE0B406038584
:10383400551190006EE0B4070385571190006FE0B6
:10384400FE900070E0C39E50030238D090006EE0FA
:10385400D39404402C90006FE0D39511500990004C
:1038640070E0C3951150028002D20290006FE0D341
:1038740095115009900070E0C395115002C2028066
:103884004990006EE0B40418900070E0C3951150A4
:1038940002D20290006FE0D395114002C202802A46
:1038A40090006FE0C395115009900070E0D395111A
:1038B40050028002D20290006FE0D395115009901B
:1038C4000070E0C395115002C202807E90006EE049
:1038D400D39404402C90006FE0C3951140099000EC
:1038E40070E0D3951140028002C20290006FE0C3E1
:1038F40095114009900070E0D395114002D20280E6
:103904004990006EE0B4041890006FE0C395115024
:1039140002C202900070E0D395114002D202802AC4
:1039240090006FE0C395114009900070E0D39511A9
:103934004002D20290006FE0D395114009900070CC
:0B394400E0C3951140028002C2022285
:093EFE002582F5825002058322A1
:10002E00EF2F500205832582F582E5833E2EF58360
:01003E00229F
:08000300C3EF9DFFEE9CFE22FD
:08003F000806B60002180622B3
:0D000E00A3E004F07006123EF4E004F022BE
:083F10000816B6FF0218162284
:0E3ED800048007C3CE13CECF13CFD5E0F62261
:103CF000BC000FBE0008ED8FF084FFADF022E4FEA3
:103D0000FF22BE000DEF60FE54F0606F20E703025B
:103D10003DA6EAC0E0EBC0E078017A0075F001EE64
:103D200020E710EF25E0FFEE33FE0AC5F023C5F0D3
:103D300030E7F0EA5407F9096A7A007B006001086D
:103D4000C3EC9E40167004ED9F4010ED9FFDEC9E6D
:103D5000FCE5F0CA4ACA03F5F08005E5F003F5F08A
:103D6000C3EE13FEEF13FFD9D77908CACBCAD8D058
:103D7000EAFEEBFFD0E0FBD0E0FA22EC8FF084FC0F
:103D8000ED54F045F0C48FF084FEEDC454F045F0DE
:103D9000C48FF084FDEEC4FE54F02DFFEE540F3CB2
:103DA000FEADF07C0022790078008FF0EC7E0820D8
:103DB000E70DC3CD33CD33C933C9C833C8DEF08472
:103DC00049F9E5F08FF0BE00E6FD7C00E9FFE8FE72
:013DD00022D0
:0E3EE600F88FF0A4FFE5F0CE88F0A42EFE22A7
:103EB800600D782B023EC2007830D8FED5E0F8229B
:103EC800EEC0E07E00123CF0EFFDEEFCD0E0FE22FA
:03000B00023E674B
:03001B00023E8220
:03002B00023E9DF5
:03000000023F07B5
:093F070075817175D0000207EA12
:0B001E00E5822FF582E5833EF583228A
:0A3EF4000582D58202158315822293
:103E6700C0E0C0F0C083C082C0D075D0001207DFA9
:103E7700D0D0D082D083D0F0D0E032C0E0C0F0C044
:103E870083C082C0D075D0001207E2D0D0D082D0D4
:103E970083D0F0D0E032C0E0C0F0C083C082C0D091
:103EA70075D0001207E5D0D0D082D083D0F0D0E013
:013EB70032D8
:00000001FF
